:040000006F00204429
:100004000000000000000000480200004A02000056
:100014000000000040040000000000000000000098
:100024004004000040040000000000000000000044
:100034004C1F00000000000040040000000000000D
:10004400400400004004000040040000400400009C
:10005400400400004004000040040000400400008C
:10006400F61900004004000040040000FC160000E3
:10007400400400004004000040040000400400006C
:10008400400400004004000040040000400400005C
:10009400400400004004000040040000400400004C
:1000A400400400005A1F0000400400004004000007
:1000B400301F0000821E00004004000040040000C5
:1000C400400400004004000040040000400400001C
:1000D4004004000040040000400400006C1D0000C7
:1000E4008E1A000040040000400400004004000098
:1000F40040040000B21D0000400400004004000061
:1001040040040000400400004004000040040000DB
:100114004004000000000000000000000000000097
:1001240000000000000000000000000000000000CB
:0C013400000000000000000000000000BF
:10014000397101436EC619A0397141536AC866CA34
:1001500062CC5ECE19A0397101535AD056D252D416
:100160004ED64AD826DA22DC06DE3301614082828E
:1001700041114AC026C222C406C68282B24D410144
:10018000024D924C224CB24B4101024B924A224A00
:10019000B2494101024992442244B2404101828065
:1001A0003D432A876373C3029377F700BDEFADE544
:1001B000937606FF3D8ABA960CC34CC30CC74CC756
:1001C0004107E36BD7FE11E28280B306C3408A0683
:1001D0009702000096966780A6002307B700A30643
:1001E000B7002306B700A305B7002305B700A30493
:1001F000B7002304B700A303B7002303B700A3028B
:10020000B7002302B700A301B7002301B700A30082
:10021000B7002300B700828093F5F50F9396850011
:10022000D58D93960501D58D61B7939627009702DA
:10023000000096968682E78086FA9680C1171D8F09
:100240003E96E374C3F8A5B701A001A0EFF25FF2F8
:100250000545EF00F03B9922EF10B068716513057A
:100260000520EF10106AB707002083A50710375547
:1002700000001305C577EF408033112DAA8537554F
:1002800000001305C578EF408032EF20C060EF20FA
:10029000805C014501B7EFF2BFED371402401C400E
:1002A0003707FF08411193E717001CC05C40F98F26
:1002B0005CC01C403707F7FE6D17F98F1CC01C404F
:1002C0003707FCFF7D17F98F1CC05C40370701FF23
:1002D0007D17F98F5CC0B7079F001CC4EF00501A50
:1002E00002C402C6B7270240054798C31C404167B5
:1002F000B7160240D98F1CC03706020005679C4222
:10030000F18F3EC6A24785073EC4B24781E7A247A8
:10031000E397E7FEB71702409C431397E700635744
:10032000070685473EC6324785476313F706B7176A
:100330000240D843B706C1FFFD16D8C3D843D8C37F
:10034000D84313670740D8C3D843758FD8C3D84361
:10035000B7061100558FD8C39843B7060001558FD3
:1003600098C3984393166700E3DD06FED843B7169B
:100370000240719BD8C3D84313672700D8C32147D5
:10038000DC42B18BE39EE7FE410129B502C661BFA5
:10039000372702401C43F19B1CC3FDB7B716024030
:1003A000DC42370700201146B18B13070710638F1B
:1003B000C70221466381C70495EB9C42918B9DC780
:1003C000B7470F00938707241CC3B7170240DC43CD
:1003D000918393F6F700B707002093870700B6973D
:1003E00094231C43B3D7D7001CC38280B7177A006D
:1003F00093870720D1BFDC42D4424166C983BD8BBD
:10040000F18E890745466393C700C94781EEB74619
:10041000024083A60680C18A89CEB7167A009386E9
:10042000062021A8B7160240D4421396E600E356F0
:1004300006FEB7163D0093860690B387D70269B7CC
:1004400001A0970100209381E14B17510020130177
:1004500061BB176500001305E584970500209385AF
:1004600065BA1386818163FAC5008322050023A043
:10047000550011059105E3EAC5FE13858181938539
:1004800081C86377B500232005001105E36DB5FE33
:10049000FD42739002BC8D427390428093028008AB
:1004A0007390023097020000938202B693E232000A
:1004B00073905230EFF03FDE97020000938242D9F2
:1004C0007390123473002030B727014093870740A0
:1004D000631FF500EFF2DFC9854513050020EF002B
:1004E000102D814513050020EF00702C65B182802E
:1004F0005C413707F1E01307F7EF944D7D8F9C4186
:10050000D58FD44DD58FD441A206D58FD98F5CC15C
:100510001C4537F7F1FF1307D77FD4457D8F9C49E2
:10052000D58F94458606D58FD98F1CC55C55370766
:1005300010FF7D177D8FDC29FD1793F7F70FD2078A
:10054000D98F5CD582801C4589C593E717001CC5EF
:100550008280F99BEDBF1C4589C593E707101CC538
:10056000828093F7F7EFE5BF1C4593E787001CC532
:10057000828008450D81058982801C4593E74700EC
:100580001CC5828008450981058982801C4591C56A
:1005900037075000D98F1CC582803707B0FF7D1701
:1005A000F98FD5BFA54763F7B7048D47138765FF5C
:1005B0003307F7020328C5009D47B397E70093C7A9
:1005C000F7FFB3F70701B396E600DD8E54C59947F0
:1005D00063E3C70495477D163306F6025859FD4775
:1005E000B397C70093C7F7FFF98F3396C5005D8EA9
:1005F00050D982800D473387E502032805019D47C6
:10060000B397E70093C7F7FFB3F70701B396E60088
:10061000DD8E14C96DBFB14763E2C7029547651609
:100620003306F6021859FD47B397C70093C7F7FF83
:10063000F98F3396C5005D8E10D9828095474D168F
:100640003306F6025855FD47B397C70093C7F7FF27
:10065000F98FB395C500DD8D4CD582806845420584
:100660004181828008416D8D3335A00082805C41DC
:1006700091C537070004D98F5CC18280370700FC21
:100680007D17F98FD5BF3C4989C593E707083CC959
:10069000828093F7F7F7E5BF3C4989C593E70704E4
:1006A0003CC9828093F7F7FBE5BF3C4993F7F7FD20
:1006B0003CC93C49DD8D2CC98280EFF27FABB70687
:1006C0006745B7270240938636123797EFCDD4C3DC
:1006D0001307B79AD8C3D4D3011198C7D45B138733
:1006E000470313962600E34B06FED45737250140F7
:1006F0001305054093E60620D4D7DC5BB70600203F
:10070000D58F1CC31C431C4537070E00D98F1CC551
:100710001C4593E717001CC53C4993E707043CC9F7
:100720001C4593E787001CC52A842285993575FDF1
:1007300037250140832785401305054093E747008F
:100740001CC52A8422853D3D75FD3725014005469F
:10075000C945814613050540B135254623040100EE
:1007600037270140B70550001C84637FF60423043B
:100770000100A54621461C8463FFF60623150100EF
:100780002304010095461C8463F1F60E38853C85F0
:1007900099460D46B3F7D702056513050580335713
:1007A000D702B3D7C702BA97C207C1837C85B727E0
:1007B000014003A78740799B23A4E7403C8505615E
:1007C0001D8D42054185F9B283278740CD8F2324B3
:1007D000F74083270740898BEDDF1C848326C744BD
:1007E00008108607AA972396D7FE1C84850793F7DF
:1007F000F70F5C8495BFA30401009C846378F60026
:100800001C84850793F7F70F5C84B5B798849C84A4
:100810000C100607850786072E97AE970357C7FE6D
:1008200083D7C7FE63FDE7029C848607AE9783D714
:10083000C7FE7C859C84988485078607AE9783D500
:10084000C7FE931717001810BA972396B7FE9C841B
:1008500038850C1085078607AE972396E7FE9C84A3
:10086000850793F7F70FDC8449BF1C841010388587
:1008700089078607B29783D7C7FEBA97C207C18395
:100880007C851C84850793F7F70F5C84EDBD03A579
:10089000C18182801C4141677917F98F1CC12320D7
:1008A00005002322050023240500B7070240232664
:1008B0000500138787006317E500D8431367F70027
:1008C000D8C382801387C7016316E500D843136736
:1008D000070FFDB7138707036318E500D843856644
:1008E000938606F0558FE9BF138747046315E5002B
:1008F000D843BD66C5BF138787056316E500D84397
:10090000B7060F00C5B71387C7066316E500D843BF
:10091000B706F000C1BF138707086316E500D84388
:10092000B706000FC1B713874709E31CE5F8D843A2
:10093000B70600F045BF1C4161773D0794517D8F9C
:100940009C45D58F9449D58FD449D58F944DD58F5B
:10095000D44DD58FD451D58F9455D58FD98F1CC1F7
:10096000DC455CC19C411CC5DC415CC582801C41EE
:1009700089C593E717001CC1828041677917F98FF9
:10098000DDBF1C4101C6DD8D0CC1828093C5F5FF22
:10099000FD8DDDBFB70702409C437D8D3335A00040
:1009A0008280EFF2EFFCFD376FF0CFFEB707024019
:1009B000C8C382805841032805004C4537060140D2
:1009C000930706403E979346F8FFB1C5832506403E
:1009D000F58D2320B640D043F18ED4C31443B3E643
:1009E000060114C3184190479346F7FF758E90C7D0
:1009F000D047F18ED4C7144541466399C600944749
:100A0000D98E94C7D447558FD8C78280B697944360
:100A1000558F98C382801C43F58F1CC38280B70713
:100A200001401387074083A70740584B698F09C7C8
:100A30007D8D3335A000828001458280B70701405B
:100A400023AAA74082809C4513F7070113F8F700FB
:100A500001C7D8413368E8008E2113F7F50F39C379
:100A600018418146854E3D4F930F800293028004CA
:100A7000214E3396DE00B3F8C50063111603939838
:100A8000260033131F011343F3FF3377E300B3183A
:100A9000180133E7E800639FF70550C98506E39A1C
:100AA000C6FD18C11307F00F6375B7045441214602
:100AB000854E3D4F930F800293028004414EB398C0
:100AC000CE0033F715016392E802131726000117D1
:100AD0003313EF001343F3FFB376D3003317E8006B
:100AE000D98E639DF701232A15010506E319C6FD7A
:100AF00054C18280E39457FA10C94DB7E39757FE6B
:100B000023281501DDB708456D8D3335A00082809F
:100B100048456D8D3335A00082800CC9828019C292
:100B20000CC982804CC98280370700C0B377E500CA
:100B30006395E708370701405C439356B501584F6A
:100B40009D8A9DE6F99BB70600FFFD16758F89C942
:100B500093160501C182D58FB706FF01758D498FA8
:100B6000B7060007D58FB7060140DCC2D8CE828019
:100B700005466396C600F59BB70680FFF9B70946A0
:100B80006396C600ED9BB706E8FFC1B70D466396B6
:100B9000C600DD9BB706FCFF4DBF11466397C6003C
:100BA00093F7F7F3B706C0FF4DB71546E391C6FAC2
:100BB00093F7F7CFB706E0FF49BF370700406391CF
:100BC000E702B7070140D84F4205B367A70089E5A0
:100BD0001345F5FFB377E500370701405CCF82800E
:100BE000A9E337080140B707300003264800131770
:100BF0000501B376F50041836396F602B70600F966
:100C0000FD16B377D60003264800F18E2322D800C4
:100C100091C5558112053315A700C98F37070140CB
:100C20005CC382809317B50063D007029357050118
:100C300093F6F7008D47B397D70093C7F7FFF18F6F
:100C4000B7060007D58FE9B7935755019207B31739
:100C5000F700E5B713F7C50F93F73500B705014067
:100C6000BA9594458A073D473317F7001347F7FFB6
:100C7000758F98C598453315F500598D88C58280C4
:100C8000EFF20FCF37F4FF1F032744723706003E01
:100C90004111931797019346F7FFF18F0607370627
:100CA0003E00718FD98F3706000113979600718F20
:100CB000D98FBD824167F98ED58F02C202C402C6A8
:100CC00023A0F182035784728545239CE18003278A
:100CD00004721305D00323A2E1820327447023AEDC
:100CE000E180412C8327447037073A1013070770BF
:100CF00093F7F7F06380E7106361F702370732106C
:100D0000130707706380E70637073710130707706C
:100D10006387E70841016FF0EFC737073B10130700
:100D20000770638BE70A37073D1013070770E393DB
:100D3000E7FE85452165CD3BB7140140E1771304FB
:100D400080044C00138504807C8222C6ED398567BF
:100D50009387C7334C00138504C07C8222C6E531DB
:100D6000F9770DA085452165C133B714014093077C
:100D700000E0130480044C00138504C07C8222C66A
:100D8000D93189674C00371501407C8222C665390C
:100D90008D477C8222C64C001385044025A8B714D9
:100DA0000140E17793870770130480044C0013859A
:100DB00004807C8222C641399307D0E34C0013851E
:100DC00004C07C8222C64131F9777C8222C64C0065
:100DD000371501408D393DBFB7140140E177130449
:100DE00080044C00138504807C8222C6A9399307B5
:100DF00040208DB7B7140140E177130480044C0004
:100E0000138504807C8222C63D398967F51799B71E
:100E100023A4A182828003A78182854714216310C5
:100E2000F7021C31639CE7023C21960793E707F821
:100E300037E700E093F7F70F36972300F7400547B1
:100E400093D756003317D700544189CE93870704B0
:100E50008A07B7E600E0B69798C38280EDF33C219D
:100E60009607F9B793870706E5B7B7160240DC4245
:100E70003747FF7F7D17F98F5D8DC8C28280371796
:100E800002405C439146B18B638CD706A146638ECA
:100E9000D706BDE71C43918BA5C7B7470F009387C3
:100EA00007241CC1371602405C4237070020130795
:100EB00007019183BD8BBA9794231C41B3D7D70008
:100EC0005CC15442A1829D8ABA969422B3D6D700BF
:100ED00014C55442AD829D8A36971423B3D6D700E9
:100EE00054C55842634C07005C42B98313F737007E
:100EF00093874180BA979C23B3D7F6021CC982809E
:100F0000B7177A009387072069BF5C435843C166CF
:100F1000C983BD8B758F8907C5466393D700C947C1
:100F200001EF3747024003270780418B09CF37176E
:100F30007A001307072021A8371702405843931659
:100F4000E700E3D606FE37173D0013070790B38787
:100F5000E70281BF99C5371702405C4B5D8D48CBD6
:100F60008280B7170240D84B1345F5FF798DC8CB67
:100F7000828099C5371702401C4F5D8D08CF828053
:100F8000B7170240984F1345F5FF798D88CF8280BF
:100F900099C5371702405C4F5D8D48CF8280B717E7
:100FA0000240D84F1345F5FF798DC8CF828099C58F
:100FB000371702405C475D8D48C78280B7170240F3
:100FC000D8471345F5FF798DC8C782801A218D67F0
:100FD00093870704B6217D8F9E21D58FD621D58F8B
:100FE000F621D58F9625D58FB625D58FD625D58FC9
:100FF000F625D58FD98F1EA19E291EA982801E217C
:1010000089C593E707041EA18280C207C18393F7B5
:10101000F7FBC207C183C5BF4EA582804A258280E7
:101020000A256D8D3335A00082801E21373701409F
:10103000130707C0C207C1836300E50237070040FA
:10104000630CE500130707406308E500371700400D
:10105000130707806316E500FA2193F7F7F8D98F95
:101060009A2593F7F7CFC207C183D98F371700406E
:101070001EA1130707809C416310E5025CD5DE21A9
:101080001EB5B7370140938707C06314F500BC2530
:101090001EB985475EA98280C207C1835EB5C5B708
:1010A0001E31D22103D86500C207C183F99BC20754
:1010B000C1831EB11E3156211A2DC207C1834207BA
:1010C00041831377C7F8518FB225F59BC20633666B
:1010D0000601D18F37360140130606C0C182631066
:1010E000C502D225DD9B03D80501D18F9225ED9B4A
:1010F00093F6F6CFD18FF22533660601D18E56A135
:10110000B71600401AAD9386068098416315D50046
:1011100058D91EB1828042074183DDBF1A31FD7765
:10112000FD17F98F1EB10358050256215E2D657714
:10113000D2211307F7CF7D8FF9772206FD17518F44
:10114000B3F70701F22103D8A500C20642073366B0
:1011500006013206D18F37360140C207130606C09A
:10116000C1824183C183631AC50071767D16F18EF9
:10117000F2251A06D18EC206C18256A1B7160040CA
:101180005AAD9386068098416315D50038C11EB1CB
:10119000828042074183DDBF1E2189C593E7170086
:1011A0001EA18280C207C183F99BC207C183CDBF44
:1011B0008357450491C52167D98F2312F504828096
:1011C000C607C583DDBF5E2501C6DD8D4EA58280C5
:1011D00093C5F5FFFD8DDDBF1E2189C593E7070887
:1011E0001EA18280C207C18393F7F7F7C207C183AC
:1011F000C5BF1E2DC207C183DD9BDD8D0EAD828074
:101200005A2DFD779387F77FF98FA205CD8FC207FF
:10121000C1835EAD8280B717004093870780631457
:10122000F5002CC18280C205C181E5BF1E294A2577
:10123000ED8F4205418189C76D8D3335A0008280D5
:101240000145828093C5F5FFC205C1810EA9828048
:10125000EFE21FF21629F577FD17F58FF621DA2553
:101260007971D58F1EA95625FD779387379FF58F06
:10127000D6212A842EC6D58F9625D58FB625D58F13
:101280005EA55E29C207C18393F7F7CFD98F5EA908
:101290006808F536B747014093870780B245631A5F
:1012A000F404A25756246547B387E702C206C186F5
:1012B000984163D20604060752244206B3D7E702D8
:1012C000130740064186B3D6E702B3F7E70292065A
:1012D000635506028E0793872703B3D7E70213F7F8
:1012E0007700B367D700C207C1831EA445616FE0D2
:1012F0007FEA925745BF0A07C1B792079387270332
:10130000B3D7E702BD8BD58FF9BF91C55E250967BD
:10131000D98F5EA582805A25F977FD17F98FD5BF41
:1013200013F7F50F85471583B395B7006319F700D9
:101330009307C500984301CED98D8CC3828089461E
:1013400093074501E318D7FE93070501E5B793C559
:10135000F5FFF98DDDB793F5F51F4EA182804A2187
:101360001375F51F82800A216D8D3335A0008280B0
:1013700013F7F50F85461583B397B6006311D702AF
:101380005A25F98F1A2101454207418381CB054532
:10139000A181B315B5006D8F3335E0008280894699
:1013A0006314D7001A29F1BF5A29E1BFEFE25FDCCD
:1013B00079711306000281450808EFE07FDE85455C
:1013C000114502C202C402C66D36854513050020D0
:1013D0004D360145593C371501409307400F4C00ED
:1013E00013050580372401407C8202C6EFF0AFE58B
:1013F00013050440EFF04F8D13050440EFF0EFAB01
:10140000AA852398A182375500001305C579EF30CE
:10141000001AB7070E003ECE0C088547130504409E
:101420002302F10202C802CA02CC02D0EFF04F8CB4
:10143000854513050440EFF00F91854513050440E1
:10144000EFF08FA5814513050440EFF04FA213057F
:101450000440EFF06F91930404402685EFF06F9104
:101460006DFD1305044037240140EFF00F91930404
:1014700004402685EFF00F916DFD37050080F532B1
:10148000130504408545EFF00FA0930500021305F6
:101490000440EFF08FA145616FE0DFCFEFE25FCD59
:1014A00039711306C0022A89AE8448088145EFE0ED
:1014B0003FCF854505453704024002C602C8593C66
:1014C00013058400EFF00FBDB72701409387C74491
:1014D0003ECA930700083ED4930700103ED69307F8
:1014E00000403ED8930700023EDA4C088D67130592
:1014F00084003EDC4ACC26D002CE02D202DEEFF0DF
:101500008FC30546894513058400EFF08FC7ED476B
:101510007C868D475C87680085473EC8EFF0BF8FAB
:10152000854513058400EFF08FC421616FE09FC6ED
:10153000EFE21FC4AA842E840565011185451305B9
:1015400005807D1402C602C802CA02CC02CE02C0C7
:1015500002C202C4393C6082373401408A851305D7
:1015600004C0FD1426C02314010023130100753CA0
:10157000A9473EC6C167938707063EC86C008947E6
:10158000130504C0FC83293E130504C085450D31B5
:10159000130504C08145B139130504C085452D39B3
:1015A0008545130504C0CD3E05616FE0BFBEEFE287
:1015B0009FBA797113064006938581861385819FB2
:1015C000EF0030289384819F138544011306400661
:1015D00093850193EF00F026930440069389819F41
:1015E0001389C1A081451385819FEF009026814515
:1015F0004A85FD14EF00F025F5F41306000281453D
:10160000080823A8090023A20902EFE07FB9854555
:10161000114502C202C402C6EFF0BF95854513050D
:101620000020EFF01F950145EFF03F843715014092
:10163000A9474C0013050580372401407C8202C66F
:10164000EFF06FC013050440EFE01FE813050440FE
:10165000EFF0AF862398A18285473ECA0C088947E0
:10166000130504402302F10202C802CC02CE02D0CC
:10167000EFE01FE8854513050440EFE0DFED854509
:1016800013050440EFE03FEC854513050440EFF0FF
:10169000AF80814513050440EFE07FFD1305044052
:1016A000EFE09FEC930404402685EFE09FEC6DFD96
:1016B0001305044037240140EFE03FEC930404405D
:1016C0002685EFE03FEC6DFD130504409546054689
:1016D0008545EFE03FED95460946130504408D45ED
:1016E000EFE05FECB165938505B8294591358945F3
:1016F0001385C182653345616FE03FA9011109453A
:1017000022CE26CC4ACA4EC852C6EFF08FA925C1B8
:10171000938521831385819FEF0070161384819F29
:10172000138A218303570A001C48930944019385B7
:101730002183998F4E859384C1821CC8EF00301499
:10174000922018485C5083560A00329718C8BA2075
:101750008E201385819FBA97958F5CD0EF00700F14
:10176000AE204E85EF00F00E0945EFF02FA4724435
:10177000E2445249C249324A056173002030EFE227
:101780003F9F011185452145EFF0AFFE854511656D
:10179000EFF01F803714014085678D447C808A8577
:1017A000C147130504C03EC426C2EFF0CFA91305FC
:1017B00004C08565EFF06FB6896761498A851305B6
:1017C00004C07C804AC426C2EFF0EFA791677C80FA
:1017D0008A859147130504C03EC4EFF0CFA6E17798
:1017E0008A85130504C07C804AC426C2EFF0AFA5E9
:1017F000B70704013EC6B70702003EC8B70700029C
:101800008507374400403ECAA1473ECC6C009D4747
:1018100013050480FC86EFF06FFB854513050480FB
:10182000EFF0EFFD05616FE0FF96EFE2DF92B74466
:1018300000402A891304900C9389048089454E85C1
:10184000EFF00FFE05C9CA8513850480B744004038
:10185000EFF08FFC1304900C1389048085454A85B2
:10186000EFF00FFC19CD13850480EFF02FFB1375FB
:10187000F50F31A07D141374F40F69F001456FE08A
:10188000DF907D141374F40F71F8CDBFEFE25F8E1B
:101890002A89371501402E84130505C08565B28459
:1018A0000146EFF0CFA70D454937135504011375D5
:1018B000F50FA53F135584001375F50FBD3713754C
:1018C000F40FA537014493170401C18363EC97001B
:1018D0003715014005468565130505C0EFF02FA4B7
:1018E0006FE05F8B1305F00F8937B307890088A37A
:1018F0000504D1BFEFE2DF87411185451145EFF0C7
:101900004FE785452145EFF0CFE6930700107C8235
:1019100037150140C1473EC64C008D471305058071
:101920003EC4EFF04F9241016FE0DF86EFE25F844B
:10193000411185454145EFF0CFE3856793870780E7
:101940007C8237150140C1473EC64C008D471305C8
:1019500005803EC4EFF02F8F41016FE0BF83EFE2BF
:101960003F81411185452145EFF0AFE0930700101D
:10197000371401407C82C1473EC64C008D47130599
:1019800004C03EC4EFF02F8C0146930500101305F0
:1019900004C0EFF0CF9841016FE0CFFFEFE24FFDC1
:1019A000797185452545EFF0CFDC9147371501402A
:1019B000FC824C0893078004130505C03ECEEFF06F
:1019C0008F8889450545EFF0EFA8914705443ED043
:1019D0000810B1473ED422D602D2EFE0BFFD9307F4
:1019E00080117C86680089475C8722C8EFF0AFC20F
:1019F00045616FE02FFA4111114522C6EFF02F82A9
:101A000085476315F5022A841145EFF02F8303C73C
:101A1000218509EFB725000081461306803E938596
:101A2000E554138501A6238981848D233244410125
:101A300073002030EFE2CFF3797185451545EFF063
:101A40004FD3856737150140FC824C08930780020D
:101A5000130505803ECEEFE01FFFB1450145EFF0D5
:101A60006F9F856705443ED00810A1473ED422D61B
:101A700002D2EFE03FF4930780137C8668008D4725
:101A80005C8722C8EFF02FB945616FE0AFF00565C4
:101A9000EFE0FFF885476314F5020565EFE01FFAF4
:101AA00083C74184B7250000850781461306803E21
:101AB0009385455B138501A52382F184C1297300B9
:101AC0002030EFE2EFEA411185452145EFF06FCA82
:101AD00085451145EFF0CFCB930700203714014027
:101AE0007C82E1473EC64C008D47130504C03EC4CE
:101AF000EFE07FF5930700084C00130504C07C82DB
:101B0000EFE07FF441016FE0EFE8EFE26FE60111F3
:101B10004D3F371400409307F01D8A85130504805C
:101B20003EC002C22314010023050100EFF0EFCFF5
:101B3000130504808545EFF02FEAC16793870706F8
:101B40006C00130504803EC8231B010002C6EFF0A1
:101B5000EFDC13050480A145EFF08FEA1305048044
:101B60008545EFF06FE3854513050480EFF04FE402
:101B700005616FE02FE2411122C42A8408414AC264
:101B80004EC006C6EF20406FB757000003A6077C83
:101B900083A6477C2A89AE89EF00D065635F050282
:101BA000B757000083A7477B1CC0B757000083A529
:101BB000C77B0840EF103072EF20C0599315050124
:101BC00037150040C18113050580EFF0CFE4B24026
:101BD00022441249824941018280B757000003A67E
:101BE000877C83A6C77C4A85CE85EF00D055E35E0F
:101BF000A0FAB757000083A7877B7DB7EFE24FD7E6
:101C0000797137140140C1472A89FC828D44C1474C
:101C10004C08130504C03ECE26CCEFE0DFE20146BF
:101C2000130504C0C145EFE09FEF85452145EFF066
:101C30004FB4854537050800EFF08FB58547FC8226
:101C40004C08E147130504C026CC3ECEEFE0BFDFD1
:101C5000894491474C08130504C0E482375400407E
:101C60003ECEEFE05FDE0C10B7070C00130504C09A
:101C70004AD03ED402D223160102EFF06FDD930763
:101C8000D0137C86680085473EC84487EFF0AF9844
:101C90000546130504C093055052EFF06FE88545E3
:101CA000130504C0EFF06FE645616FE0AFCEEFE2E1
:101CB0002FCC797137140140930700022A89FC82E6
:101CC0008D44C1474C08130504C03ECE26CCEFE03E
:101CD0009FD70146130504C093050002EFE03FE4DF
:101CE00085452145EFF0EFA8854537050400EFF065
:101CF0002FAA93070040FC824C08E147130504C05B
:101D000026CC3ECEEFE03FD4856793870780FC82E8
:101D10004C089147130504C03ECE37540040EFE015
:101D20009FD20C10B7070C00130504804AD03ED494
:101D300002D223160102EFF0AFD1930770137C8615
:101D400085475C87680085473EC8EFF0CF8C054625
:101D50001305048093055052EFF08FDC8545130581
:101D60000480EFF08FDA45616FE0CFC2411122C6E7
:101D7000375400409305505213050480EFF04FDFB5
:101D80000DC513050480EFF08FDD9375F50F238AE1
:101D9000B18203A581851C4D104954498507B3E7DD
:101DA000C7026384D70031053926324441017300EC
:101DB0002030411122C6375400409305505213057C
:101DC00004C0EFF0EFDA0DC5130504C0EFF02FD912
:101DD0009375F50F238CB18203A5C1851C4D104965
:101DE00054498507B3E7C7026384D7003105E1246E
:101DF0003244410173002030EFE28FB70111AA8411
:101E00002E8409458545EFF0AF98E0843704004003
:101E10004C081305044026CA231E0100231D01009F
:101E2000EFF0AFA0130504408545EFF0AFC10546C4
:101E3000854513050440EFF00FB99307D0027C8667
:101E40008D475C87680085473EC8EFE0DFFC056191
:101E50006FE04FB4EFE2CFB1B707002083A50710C2
:101E6000896793870771B3D5F502A9473305F50252
:101E7000FD15C205C1817D1542054181B53F6FE069
:101E80006FB1411122C63704004085451305044057
:101E9000EFF0CFB919C5854513050440EFF08FBAAF
:101EA00091233244410173002030EFE26FAC011105
:101EB0002E84AA8485450545EFF08F8D4C083705A3
:101EC000004026CAE084231E0100231D0100EFF01C
:101ED000CF950546854537050040EFF0CFAE930717
:101EE000C0027C8689475C87680085473EC8EFE072
:101EF0009FF2854537050040EFF00FAA05616FE0BE
:101F00006FA9EFE2EFA6B707002083A50710896746
:101F100093870771B3D5F502A9473305F502FD157F
:101F2000C205C1817D154205418141376FE08FA611
:101F3000854537050040EFF06FAF19C5854537057A
:101F40000040EFF02FB0D12873002030B7F700E049
:101F500023A20700D92073002030411122C6373454
:101F600001408545130504C0EFF04FAC01CD1305CA
:101F700004C08545EFF00FAD375500001305057D12
:101F8000EF20207432444101730020301DC9B29605
:101F9000C206C18252A136A10CC509EE85471CA11B
:101FA00083A6C1839387C183368701EB54C588C359
:101FB0000145828023000500E5B76306A700584766
:101FC000EDB77D558280054582800DC583A7C1830D
:101FD0001387C18399E305458280D4476396A600A1
:101FE0005845D8C7014582806394A70014C3DDBF5C
:101FF000B687CDB77D558280EFE28F9703A4C1836A
:1020000075DC1C2093F7F70F99C75E2099C3230056
:1020100004001C4482974044E5B783A7C18305466A
:1020200091E38280D62381CEBA237D174207418374
:10203000BAA3BA234207418319E390A3B6A3DC47AE
:10204000C5B7232605000CC150C123240500054552
:102050008280584550411C4505073367C702630E0F
:10206000F70054455C45184186068507B3E7C7026B
:1020700036970EA35CC50545828079558280184548
:102080005C456300F70218451C410607BA979E237A
:1020900058419EA11C458507B3E7E7021CC50545CD
:1020A000828001458280232605000CC150C1232473
:1020B0000500054582805C45544118458507B3E716
:1020C000D702638EE70058451C41BA978CA35C4544
:1020D00058418507B3E7E7025CC50545828079551D
:1020E0008280B707002083A707100967130707F44A
:1020F000B3D7E702C207C1832391F1842390F1840F
:102100008280EFE2EF862A84116501118545110571
:10211000EFE03FE6930700207C82371501408D47B2
:102120003EC44C00E147130505803EC6EFE0BF9179
:1021300022C837440140B70708000C081305048083
:102140003ECC02CA231E0100EFF08F908545130597
:102150000480EFF08F9B05616FE0CF83EFD2BFFF6C
:10216000B7440140AE8932890144938404806345B9
:1021700024014A856FE06F81930500042685EFF006
:102180008F9E7DD9B3878900838507002685050446
:10219000C205C181EFF02F9CD9BF138781801C43FA
:1021A000938681C83E95636BD500B7560020938611
:1021B000068063E5A60008C33E858280FD57EDBF1B
:1021C0000397018381472A97634F070009CD05666E
:1021D0009306F6FFB6876358C700AA876305D50044
:1021E00093170701C1833E858280EFD2DFF641114C
:1021F00037240140AA894400130901011304044053
:10220000CE85228595460546EFE0CFB985452285E6
:10221000EFE0CFB789452285EFE0CFC465DD2285A9
:10222000EFE0CFC342054185613F8AA08904E319ED
:1022300099FC1547814735A01396170014088507A8
:102240003696080893961700AA96835546FF03D53D
:1022500046FF6376B500231AA6FE239AB6FEC20790
:10226000C183E3CBE7FC7D1771F728843C854101EE
:102270003E954205418105816FD03FF1EFD25FEF7E
:1022800003A581A0930740063355F5024205418519
:10229000053FEF109071B757000083A5077EEF1040
:1022A00090036FD03FEFEFD2BFEC09453D3FEF10F9
:1022B000D06FB757000083A5877FEF10D0016FD094
:1022C0007FEDEFD2FFEA03A5C1A193074006335586
:1022D000F50242054185ED35EF10306DB75700002E
:1022E00083A5077EEF10207F6FD0DFEAEFD25FE893
:1022F0001145E53DEF10706BB757000083A5877F50
:10230000EF10607D6FD01FE9EFD29FE61945F13DD8
:1023100095679387C77F01479306100F92236369E0
:10232000C5023A85EF10C037B757000003A6877E75
:1023300083A6C77EEF006077B757000003A6077F2C
:1023400083A6477FEF00F041EF10D07D6FD09FE470
:1023500005078907E314D7FC13050000C5BFEFD2BA
:102360003FE139716800130620038145EFF00FD279
:10237000188693073005370500206317F702988603
:102380009307C0046312F7020347D103D947631DC3
:10239000F700130620036C0013050502EF2000165A
:1023A000054521616FD01FDFB707002003C7470530
:1023B000130505029387470518A1983318B1B82370
:1023C00038A1B83338B1D82358A1D83358B1F8233D
:1023D00078A1F83378B19827DC3718A5A308F5025F
:1023E0000145C1B7EFD2DFD8513D138401A2935705
:1023F000850048B87CA89357050161817CB808AC7A
:10240000C9359357850008BC3CAC935705016181E1
:102410003CBC48AC493D9357850048B47CA49357D5
:102420000501618108A868287CB45C382205B7647E
:1024300000005D8D7C3883A5049E37690000C207CB
:10244000C98F082C62055D8DEF10E068EF10704AAF
:10245000AA851305899EEF20801568245C3483A526
:10246000049E22055D8D7C34C207C98F0828620551
:102470005D8DEF104066EF10D047AA851305899E49
:10248000EF20E012282C1C3C83A5049E22055D8DC4
:102490003C3CC207C98F482C62055D8DEF10A063DC
:1024A000EF103045AA85376500001305C59EEF2063
:1024B00000106FD03FCEEFD2BFCB938741859843BA
:1024C000D566938606186307D702050798C33714A5
:1024D0000140856493850480130504800546EFE080
:1024E0000FE401469385048013050480EFE02FE399
:1024F0006FD05FCA23A00700B707EFBE37E700E041
:10250000938707083CC7E1B7EFD29FC693875184F2
:10251000902337140140930500101336160013055D
:10252000048090A3EFE0AFDF1387D1841C238507DD
:1025300093F7F70F1CA329476399E7000546930516
:102540000010130504C0EFE08FDD6FD0BFC4138708
:10255000E1841C233706002013060602850793F743
:10256000F70F1CA38346C6028345B602A206CD8E92
:102570006391D704EFD2DFBF138401A6138501A6B0
:102580002300070023890184EFF03FA42300040007
:10259000371401409145130504C0EFE0CFD601E99F
:1025A000014693050010130504C0EFE04FD76FD02C
:1025B0007FBE8280EFD2DFBB03C7218585471384AE
:1025C000F184938441846310F702138901A5138574
:1025D00001A5230004002398018423800400EFF068
:1025E000DF9E23000900982085476315F7001C2013
:1025F00085071CA0370900209306090283C7E6025D
:1026000003C6D6021420A207D18F130909026390D2
:10261000F60223000400138401A5138501A523807D
:102620000400EFF09F9A230004006FD0BFB68547E7
:1026300063FDE700371501400146930500101305BF
:1026400005C0EFE0CFCD230004003715014093050E
:102650000010130505C0EFE0AFCB9387018501E5BE
:102660009A2305079AA3034709030346F902962311
:102670002207518FE39BE6FA371501400546930583
:102680000010130505C023900700EFE04FC961B7A4
:10269000EFD27FACB70400209384040283C72402E6
:1026A00003C51402A2075D8DEF103030B76700003C
:1026B00083A5079E138401A2EF10A005BC20938977
:1026C0008184370700203CA0BC30130747052380D6
:1026D00001A23CB0DC20A38001A223A0A9005CA041
:1026E000DC30138901A25CB0FC207CA0FC307CB003
:1026F0009C241CA43C271437A207D58F1CB4A183AB
:102700003CA45C273437A207D58F3CB4A1835CA4DA
:10271000EFF07FB99357850048B47CA49357050127
:1027200061817CB408A8EFF07FB59357850048B865
:102730007CA89357050161817CB808ACEFF07FB8A5
:10274000935785015CAC7C24443413578500A20761
:10275000C58F643438AC13570501C204C58F0428F3
:1027600038BC5838E204DD8C7C28AA8508BCA20756
:102770005D8F7C38C207D98F182C62073365F7004C
:10278000EF10A05E83A50900EF10E034AA8526852E
:10279000EF10A05D9357850008B83CA8935705013A
:1027A00061813CB848A8EFF07FB493578500A3003F
:1027B000A4022301F402935705016181A301F402ED
:1027C0002302A402EFF05FB4935785002303F402C1
:1027D00093570501A303F4023C280438A302A40282
:1027E000A207C58F243861812304A402C204C58FC7
:1027F0004428E204DD8CB767000083A5C79F2685C7
:10280000EF10A024634B0500B757000083A5877F16
:102810002685EF10201B6355A00005472386E18421
:10282000B714014093050010138504C0EFE04FAECC
:10283000814701C99145138504C0EFE0CFACB337A0
:10284000A000A304F90223050902A3050902230637
:1028500009026FD09F93EFD2BF91EFF05FB0EFF01E
:102860003FE3B725000081461306803E93858550DF
:10287000138501A7EFF08FF1B7250000F946130685
:10288000803E9385654B138501A8EFF02FF0EFF0A4
:10289000AFF66FD03F90EFD2BF8D0545EFF06FE6FA
:1028A0009128EFF08FA6EFE07FB0EFF0AF84EFF06C
:1028B000EF87EFE0DFECEFF08F8AEFF02F8EEFF095
:1028C0006F97EFE0DFCE1305C012EFF0AFD83705FA
:1028D0000040854513050540EFE01F8CB7670000F9
:1028E00083A707A023A6F1801385C180EFF0AFA8CE
:1028F0006FD05F8AEFD2DF873704002013044406CD
:102900001306800C938501A91305C400EFF0AFF9FD
:10291000716513050520EFF08FB9854404A01306F7
:10292000C012938581B51305840223AC8184EFF036
:102930008FF748507104EFF06FAC04A0014523AE4F
:1029400081846FD03F8513D74501B7071000FD176D
:1029500013D846011377F77F9308F07F33F3B7005E
:102960002A8EF58FFD81B28E1378F87FFD82630881
:102970001703630018030DEBB368A300631408008A
:102980005D8E29CA638508046388D502054595EDE7
:102990008280B3E8C700E38008FE79558280336502
:1029A000A30065FD630CE802631408005D8E79DE08
:1029B000E39ED5FCE34CE8FC63480701E3E867FCD1
:1029C0006303F302637FF30081E57D558280F5DECA
:1029D000054582800145E39B08FA82805D8E69DAB5
:1029E0006DBF01458280E3E3CEFB0145E372DEFB70
:1029F000E5F1E1BF13D74501B7071000FD1713D864
:102A000046011377F77F9308F07F33FEB700AA8E55
:102A1000F58FFD81328F1378F87FFD82630E1703E7
:102A2000630D180129E3B368AE00631F08005D8ED3
:102A300001EE0143638C080421A8B3E8C7000943F1
:102A4000639608046DD305A0638408046385D502EA
:102A500005438DCD7D531DA8B368AE000943639730
:102A60000802630AE802631408005D8E75D2E391E0
:102A7000D5FEE34FE8FC63490701E3EBC7FD630FB5
:102A8000FE0001436374FE00F1D505431A85828080
:102A9000EDFE7D53E5BF5D8E79DACDBFE36ADFFBE6
:102AA0000143E3F5EEFFF5F175B739714AD813D953
:102AB00045014ED652D456D29399C50006DE22DC8B
:102AC00026DA5AD05ECE1379F97F2A8A93D9C900C3
:102AD00093DAF501630D090E9307F07F6306F91889
:102AE0001354D5018E09B36934013704800033E4EF
:102AF000890093143500130919C08149814B13D7FC
:102B00004601139AC6001377F77FB285135ACA009D
:102B100013DBF601630B07109307F07F6303F704E1
:102B20009357D6010E0A33EA4701130717C0B707B8
:102B30008000B367FA00931536003A99814833C78D
:102B40006A01BD463A851308190063E8361717363F
:102B50000000130666EB8A09B29983A60900B296B3
:102B60008286B367CA001309F97F6399071293E954
:102B7000290081458948E1B701479307F07F370471
:102B8000080081443204D20731807E075D8C598C65
:102B9000A285F250625426854259D254B259225A23
:102BA000925A025BF24B216182805A853E84AE8448
:102BB000C68B8947638DFB0E8D47E38FFBFA8547F4
:102BC0002A87639EFB3881470144814465BF33E413
:102BD000A90061C036C632C4638C092A4E85EF1045
:102BE000100B2246B246AA87130755FF75449384FB
:102BF00087FF198CB399990033548A0033643401E8
:102C0000B3149A0013D746011309D0C0139AC60013
:102C10001377F77F3309F9408149814BB285135A05
:102C2000CA0013DBF601E31907EEB367CA00B1C7A8
:102C3000630F0A22528532C4EF10700522462A879C
:102C4000930655FFF547930587FF958F331ABA0012
:102C5000B357F600B3E74701B315B6003309E940AF
:102C60001309D9C08148E1BD33E4A90001ECA149B1
:102C700081441309F07F894B59B593E919008145C7
:102C8000854875BD4E84AA84B1491309F07F8D4BE8
:102C9000BDB5914981440149854B95B593E939000A
:102CA000D2878D4869BD89475685E397FBF02A870F
:102CB0009307F07F01448144F1B5C16E1386FEFF96
:102CC00093D6040113DE0501F18CF18D3386950254
:102CD0003383B6029358060133059E021A95AA98CB
:102CE000B382C60363F36800F692C16F1383FFFFDC
:102CF00033F5670093D30701B3F76800C207337356
:102D000066003E933306950293D80801B387A60266
:102D1000135F0601B3849302BE94FA94B38E7602D5
:102D200063F3F400FE9E416A9307FAFF935F040188
:102D3000B376F400B3F9F4007D8EC1803384D502FC
:102D4000C209338FD401B299CE98B307DE02935EE5
:102D50000401B385BF02AE97BE9E330EFE0363F33C
:102D6000BE00529EC1679385F7FF33F6BE006D8C9F
:102D70004206229693DE0E01B305D502769E338578
:102D8000AF0213D40501B386D302AA96A296B38FDD
:102D9000F30363F3A600BE9F41657D15B3F7A6005C
:102DA000C2076D8DAA97B3855800B3B93501FA975C
:102DB000B2953384370133B6C500B30EC4013385F1
:102DC000CE0033343401B3B7E701C18F33BECE0137
:102DD00013D406013336C5003E943366CE00939477
:102DE000950032947E94B3E46400260493567501F2
:102DF000B3349000DD8193179500CD8C558CDD8C1C
:102E00009317740063DB070093D71400858893162B
:102E1000F401DD8CD58C058042899307F93F635915
:102E2000F00893F6740081CE93F6F400114663889F
:102E3000C60093864400B3B496002694B6849316D5
:102E4000740063D80600B70700FFFD177D8C930759
:102E500009409306E07F63CFF60E93D634009314B7
:102E6000D4012604D58C318093F7F77F21BB3285BE
:102E700032C4EF10C06193065501F14713070502F4
:102E80002246E3D1D7DC6115B317A6008145F9B31B
:102E9000EF10E05F13075501F14593070502224645
:102EA000B246E3D5E5D461153314AA00814499BB39
:102EB00085469D8EB1E71309E941B3972401B3D448
:102EC000D40033192401B337F000B3649900DD8CCA
:102ED00093F77400B356D40081CF93F7F4001146F2
:102EE0006388C70093874400B3B49700A696BE8456
:102EF0009397860063D8070485470144814459B1FC
:102F000013068003E341D6CC7D46E356D6FA055638
:102F1000B307F640930500023356F4006387B6000A
:102F20001309E943B3172401DD8CB3349000D18C2D
:102F300093F67400014499CA93F7F4001146814650
:102F4000E392C7FA139496003180F6068D80D58CF3
:102F500081470DB99307F07F0144814425B142892F
:102F60006DBD370710007D1701113373B70093D87B
:102F70004601758F935ED60122CC26CA0E0393D4E8
:102F800045019357D5010E0706CE4AC84EC693F8A1
:102F9000F87F130EF07F33E7EE0093F4F47F13D441
:102FA000F50133E36700131F3500FD82931E3600E1
:102FB0006380C81993C61600B38514416305D41203
:102FC0006351B018638B081AB70780005D8F638167
:102FD000C4599307800363C4B734FD4763C5B7483A
:102FE000930700028D8FB3D9BE003318F700B39E4C
:102FF000FE00336838013357B700B339D001336866
:1030000038013303E340B3090F41B3373F013306BF
:10301000F3409317860063D30724370980007D1996
:1030200033792601630F092C4A85EF1040461307B8
:1030300085FF93070002998FB3D7F9003316E90093
:10304000D18FB399E9006344972A058F13061700BF
:10305000FD4663C5C63A13070002118FB3D6C900F7
:103060003398E9003397E700558F33380001B3698F
:10307000070133D6C700814493F7790081CF93F6D7
:10308000F90091476388F6009386490033B836010A
:103090004296B6899317860063D6071C13871400DF
:1030A0009307F07F05886306F720B70780FFFD17B9
:1030B000F18F1398D70193D93900A60733683801E7
:1030C000B1831377F77F9396C7005207B1827E04CE
:1030D000D98EC18EF2406244D2444249B2494285FF
:1030E000B685056182806356B00A638A0812B70705
:1030F00080005D8F6387C42D9307800363C7B71873
:10310000FD4763D2B73C138805FE93070002B3590D
:103110000701638AF50093070004B385B7403317AE
:10312000B700B3EEEE003338D0013368380195A212
:10313000B367D7019385148099E393C61600630A99
:10314000D404D1E19387140093F7E77F6399071EB6
:10315000B367E3013368D701639204166382073CC7
:1031600063160842131835009316D301135838001C
:1031700033E806019357330019A2B367D70163857B
:10318000071A9387F5FF638B073A638CC523BE85C7
:1031900089B56399051C9386140093F7E67FC1EF08
:1031A000B367E30163900436638D0744B367D701C7
:1031B000639407460E051318D3010D813368A800E8
:1031C000935733006DA8B385984063970420B36785
:1031D000E301638D07309387F5FF6389074013058B
:1031E000F07F6383A520BE859307800363C2B72A5F
:1031F000FD4763C8B73C930700028D8F3318F30077
:103200003356BF00B317FF003368C800B339F0006E
:103210003353B3003368380133076740B5ACB36745
:10322000D701638307109387F5FF638F071E6380C1
:10323000C52FBE85D1B59307F07F638BF606FA9E46
:1032400033B6EE01B307E300B2971398F70193DEAC
:103250001E00B369D80113D61700B68493F779001E
:10326000E39F07E09317D60113D839003368F800BD
:10327000A685935736001307F07F6380E506B207F3
:10328000B18313F7F57F05883DBD3367D701333828
:10329000E000B309E801B3B7E9013386670093178B
:1032A0008600E3DD07FA85049307F07F639CF4183A
:1032B00005881307F07F8147014831B563910710F6
:1032C0006301083C131836009317D70113583800D0
:1032D0003368F800368493573700B367F800E9DBAA
:1032E00001441307F07FB70708000148E9BB370620
:1032F00080FF7D167D8E93F77900998CE39107D836
:1033000095B74E85EF10A01813078501FD47E3D24E
:10331000E7D2130685FFB397C90081492DB33368FF
:10332000D70133380001C5B1131835009317D30105
:10333000135838003368F800935733002DBFB30992
:10334000DF413309E34033363F013309C940931766
:10335000890063CA072033E82901E31508CC8147B7
:10336000014431BFB385984063810414B7068000DF
:103370009307F07F3363D3006381F82093078003C2
:1033800063CCB722FD4763C9B72C930700028D8F2A
:103390003318F300B356BF00B317FF003368D800EB
:1033A000B339F0003353B300336838011A97B309C7
:1033B000D801B3B7D9013386E700C684CDB5E31190
:1033C00008F2131835009317D301135838003368E7
:1033D000F8009357330011B7370580009307F07F4B
:1033E0003363A300E392F8E00E061318D7010D82B1
:1033F0003368C800935737003684C5B50517930660
:10340000000233D7E700630AD60093060004338630
:10341000C6403396C700B3E9C90033383001B369F9
:10342000E800014681441DBDB309DF01B307E30095
:1034300033BFE9013386E701931786008544E3DF54
:1034400007E08944B70780FFFD17F18F13D71900F4
:1034500013F81900336807019399F701B3E90901DB
:1034600013D6170011B9138805FE93070002B3594C
:103470000701638AF50093070004B385B74033174B
:10348000B700B3EEEE003338D00133683801A5BE83
:103490003363E30133386000B3890E41B3B73E01B3
:1034A0003306F740C6843684ADB6B367E30163875D
:1034B00007189387F5FF638C071C9306F07F638ED4
:1034C000D50ABE8565BD930700028D8FB3D9BE00B6
:1034D0003318F700B39EFE00336838013357B70046
:1034E000B339D001336838013A9365B31318360005
:1034F0009317D7011358380033E8070136849357E0
:10350000370095BBBDCB3367D701E31B07DC0E0546
:103510001318D3010D813368A8009357330075BB8E
:10352000E30F08E2131836009317D7011358380039
:103530003368F80036849357370091B3B309DF41FD
:10354000B307E340333F3F013386E7418544D1B4BD
:10355000131835009316D3011358380033E80601C9
:10356000935733009DBBB389EE413306674033B9AF
:103570003E0133092641368475B40E061318D7016F
:103580000D823368C8009357370081BBB309DF4110
:10359000B307E34033363F013386C74093178600B5
:1035A00063D7070AB389EE41B3076740B3BE3E0154
:1035B0003386D7413684C9B43363E30133386000BE
:1035C000FDB3138805FE93070002B3590301638A14
:1035D000F50093070004B385B7403313B300336F8E
:1035E0006F003338E001336838017DB5B389EE41AF
:1035F000B3076740B3BE3E013386D7413684854466
:1036000009BC131836009317D701135838003368D4
:10361000F80093573700A5B1B309DF01B307E30002
:1036200033BFE9013386E70193178600E3D807C269
:10363000B70780FFFD177D8E85440DB10E06131868
:10364000D7010D823368C800935737002DB133E896
:10365000C900E30608D019B1138805FE93070002DC
:10366000B3590301638AF50093070004B385B7409B
:103670003313B300336F6F003338E0013368380120
:103680003DB301441307F07FB70708002DBCB30911
:10369000DF01B307E300B3BED9013386D70169BBAD
:1036A000411106C622C426C20DCD9357F541B3C4BD
:1036B000A7009D8C2A842685EF00705D9306E0416B
:1036C000898EA9477D8093F6F67F63CDA7022D47AB
:1036D000098FB3D7E4005505B207B394A400B183B2
:1036E00029A00144814681478144B207D206B183B3
:1036F0007E04D58FC18FB24022442685BE85924478
:10370000410182805515B397A400B207B18381446B
:10371000E9BF3971935775014AD856D25ECE931AD4
:1037200095001359F50106DE22DC26DA4ED652D476
:103730005AD093F7F70F93DA9A00CA8B6382071275
:103740001307F00F6384E7128E0A37070004B3EA09
:10375000EA00138A17F80144014B93D7750193943B
:10376000950093F7F70FA58093D9F501FDC71307CF
:10377000F00F6387E7028E04938717F8370700047A
:10378000D98C330AFA408146558C1727000013075D
:10379000A72B0A043A941C4033493901BA9782870F
:1037A000130A1AF0F9E88946558C17270000130709
:1037B000A72D0A043A941C4033493901BA978287ED
:1037C00001491307F00FB707400013959700F25017
:1037D00062549317770125817E095D8D336525013C
:1037E000D2544259B259225A925A025BF24B216189
:1037F00082801307F00F8147C9BFA68ACE8B368B14
:103800008947630BFB1A8D47E30CFBFA8547630A74
:10381000FB0A1307FA0713F91B006357E01293F72B
:103820007A0099C793F7FA0091466383D700910A0B
:1038300093974A0063D90700B70700F8FD17B3FA5A
:10384000FA0013070A089307E00FE3C4E7FA939717
:103850006A00A5831377F70F8DBFB9E48546A9B732
:1038600063940A021144014A054BC5BD63990A00DD
:103870002144130AF00F094BCDB58D4631B73144C1
:10388000130AF00F0D4BD1BD56852EC6EF00304008
:103890009307B5FFB39AFA009307A0F8338AA740BD
:1038A0000144014BB24555BD2685EF00503E13073C
:1038B000B5FFB307AA00B394E400138A67078146F3
:1038C000E1B513F91B000147814701B74166139524
:1038D00054007D1693570501698E63FA9A0AB3D591
:1038E000FA027D1AD68601473388C502B3F6F6027E
:1038F000C206558F637B07012A979386F5FF63689D
:10390000A70A6376070BF9152A9733070741B356C1
:10391000F7023377F702B38AC6029317070163FBF6
:103920005701AA971387F6FF63E1A70863FF5707BC
:10393000F916AA97C205B38A5741D58DB33A5001FB
:10394000B3EA5501CA8BF1B58546998E11C76D460C
:1039500001478147E34BD6E6130AEA09339A4A0145
:10396000B3D7DA00B33A4001B3E7570113F7770052
:1039700019C713F7F70091466303D7009107139710
:103980005700634807029A07A58301473DBD93D6B8
:103990001A00B3D5F6021397FA0141833388C502A2
:1039A000B1B7CE8B368B814AA1BDBA8661B7B685D9
:1039B000A9BF0547814711BD13F91B001307F00F7D
:1039C000814721B593567501B7078000FD1713D6BF
:1039D000750193F6F60F1308F00FB3F8A70013570D
:1039E000F501ED8F1376F60FFD8163810603630CFD
:1039F00006018DE211E2B1C3638E08026305B704CC
:103A000005451DE78280F5D779558280E39E08FE43
:103A10006309D60211E2EDD7E314B7FEE342D6FE06
:103A200063C7C600E3EE17FD0145E3FDF8FC01E7BF
:103A30007D558280F5DD054582800145E39208FCD5
:103A40008280F9DBD1B78146E1BF93567501B70794
:103A50008000FD1713D6750193F6F60F1308F00FCB
:103A6000B3F8A7001357F501ED8F1376F60FFD811C
:103A7000638706036309060185EA11EA89EB0145BC
:103A8000639B080082800945F5FFE5DA31A8638C65
:103A900008026300B704054575D77D558280094546
:103AA000639808026304D60211E2F5D7E315B7FE66
:103AB000E343D6FE63C7C600E3EF17FD0145E3F31A
:103AC000F8FC19E3D9BFF1D905458280E5D382809E
:103AD00082808146C5B7797122D4135475014ECEC8
:103AE00052CC9319950006D626D24AD056CA5AC847
:103AF0001374F40F93D99900135AF50169C493070D
:103B0000F00F6308F40E9397390037070004B3E908
:103B1000E700130414F88144014B13D77501939AFD
:103B200095001377F70F93DA9A0013D9F50145CF73
:103B30009307F00F630CF7028E0A130717F8B70705
:103B40000004B3EAFA003A94014633452A01BD471E
:103B5000AA869305140063E2971017270000130745
:103B6000A7F68A04BA949C40BA9782871304F40F8C
:103B700063980A0C93E424000946C1BF014513076A
:103B8000F00FB7074000B2502254A6075E07A58386
:103B90007E05D98F92540259F249624AD24A424B69
:103BA0005D8D45618280CA86D689328B89476301E3
:103BB000FB0A8D47E304FBFC854736856312FB1A3D
:103BC00001478147C9B7639E090413D77501939ACA
:103BD00095001377F70F91440144054B93DA9A004F
:103BE00013D9F50131F7639D0A0093E414000546EB
:103BF000A9BF63930902A1441304F00F094B31BF1D
:103C00005685EF00D0089307B5FF098CB39AFA00E8
:103C10001304A4F8014615BFB1441304F00F0D4B73
:103C2000EDBD4E852EC6EF0090069307B5FF130439
:103C3000A0F8B399F900098C8144014BB245F1BD5C
:103C400093E434000D4611B78947D286E313FBF69F
:103C500036851307F00F81473DB741639306F3FFA5
:103C600013D6090193D80A01B3F7D900B3FADA00E1
:103C700033885703B389F80213570801B30A560370
:103C8000D6994E9733061603637357011A96C16788
:103C9000FD17B376F7003378F800C206C296939901
:103CA000660093570701B3393001E982B2979A074A
:103CB000B3E6D900B3E9D7009397490063D9070069
:103CC00013D7190093F71900B369F7002E8413076F
:103CD000F4076350E00493F7790099C793F7F9006C
:103CE00091466383D70091099397490063D90700F0
:103CF000B70700F8FD17B3F9F90013070408930795
:103D0000E00F63CBE70493976900A5831377F70F60
:103D10009DBD8547B386E74011C76D460147814782
:103D2000E343D6E61307E4093397E9003337E000AD
:103D3000B3D7D900D98F13F7770019C713F7F70056
:103D400091466303D700910713975700634C070010
:103D50009A07A583014705BD1307F00F814725B5D5
:103D60002E84B5B70547814739BD3707800041111B
:103D70007D179356750113D87501B377A70093F695
:103D8000F60F935EF5013376B70026C24AC013786A
:103D9000F80F06C622C41303F00F3E8E3689F68450
:103DA000139F3700FD8113153600B3880641630267
:103DB000681093C51500638CBE106354100D63101A
:103DC00008106304051EFD18B307AF4063860802A0
:103DD0009307F00F6388F616ED4763C7172913079B
:103DE0000002330717413317E500B3571501333786
:103DF000E000D98FB307FF40139757006351071AAC
:103E0000370400047D147D8C228551256D15B31770
:103E1000A400634E251B3305254113041500130729
:103E20000002018F3397E7003337E000B3D78700F4
:103E3000D98F014913F7770019C713F7F700914697
:103E40006303D700910713975700635E0714930627
:103E500019001307F00F93FE14006386E6169A0705
:103E6000A58393F6F60FA607B240224413D5970018
:103E7000DE069397FE01558D924402495D8D410106
:103E800082806392080A138716001377E70F631B7B
:103E900007146394062263020F2071D5B307AF4065
:103EA0001397570063550722B307E5410149AE84D4
:103EB00051B7E30005F0638ABE0AE35410FD93078F
:103EC000F00F6381F608B70700045D8D31B7635EBC
:103ED0001009630108089307F00F6385F606B7071A
:103EE00000045D8DED4763C0171F13070002330701
:103EF00017413317E500B35715013337E000D98F69
:103F0000FA9713975700635C070805091307F00F2A
:103F1000630BE90AB706007E13D71700FD16858BE1
:103F2000758FD98F01BF3307D84063950610630D95
:103F30000F147D176303071A9307F00F6314F8102B
:103F4000AE84328E630F0E06814E9306F00FB707D4
:103F5000400011BF39C9FD18B307AF00E38308FA69
:103F60009307F00FE390F6F8F1BF639908081389FF
:103F700016001377E90F63160712639B061063039D
:103F80000F16E30205EEB307AF0013975700014980
:103F900063570700370700FC7D17F98F054913F7B2
:103FA0007700E31C07E813DE37009307F00FE30BFD
:103FB000F9F893179E00A5839376F90F93FE1400EA
:103FC0005DB593FE14009306F00F814769BD370776
:103FD00000FC7D17F98F13F777003309A940E31E22
:103FE00007E4D1B73304AF409317540063C3070C01
:103FF000E31C04E0814E81468147B5B53307D840C4
:10400000B5C69307F00FE30EF8F2B7070004336F5D
:10401000FF00ED4763CDE70C93070002998FB317BC
:10402000FF003357EF00B337F0005D8FB307A700F1
:104030004289C1BD9307F00FE304F8F0B70700040D
:10404000336FFF00ED4763C2E70893070002998FC3
:10405000B317FF003357EF00B337F000D98FB30722
:10406000F5404289AE8449BB854769B3630E0F06AC
:104070007D17B307AF004289E30507E89307F00F08
:10408000E319F8F8328E7DBD328E4289AE8431BF9D
:10409000E3090FEAE30805EA45BD0DCDAE8EB28710
:1040A000D9B39307F00FE300F9F2B307AF008583AC
:1040B000FDB53304E541AE8481BBE31D0FFCE30590
:1040C00005E8AE84BDBD854725BD854749BF01498B
:1040D000E39707EC814E814779B3B307E541428905
:1040E000AE8419BBB28741B3328E42897DBD05478C
:1040F00035BF37068000135775019307F6FF137716
:10410000F70F9305E007B3F6A7009357F50163FC9B
:10411000E5009305D00963FAE500370500801345F3
:10412000F5FF3E9582800145828093055009D18E2E
:1041300063CDE500130660093307E64033D7E60098
:104140003305E040F5F33A8582801307A7F63397ED
:10415000E600FDB713577501370680009307F6FF99
:104160001377F70F9305E007B3F6A7009357F50110
:10417000014563F4E50099C3828082809307E009DA
:104180007D55E3EBE7FE93055009B3E7C60063D71F
:10419000E5001307A7F63395E70082801305600951
:1041A0003307E54033D5E7008280411106C622C4BB
:1041B00015CD2A84E92C9307E0093387A74093079C
:1041C000600963C0E704A1469377F70F63D5A600A3
:1041D00061153314A4002604258026041355940089
:1041E000B2402244DE075D8D4101828001442604F5
:1041F00013559400B24022448147DE075D8D410192
:1042000082809307900963DDE7009307B501954627
:10421000B317F400898EB337F0003354D4005D8CAB
:10422000954763D6A7009307B5FF3314F400B7068C
:1042300000FCFD16937774003376D40085C3937722
:10424000F4009145638CB70011069317560063D7AD
:1042500007009307F009758E3387A7401314660093
:104260002580260413559400B24022449377F70F1B
:10427000DE075D8D41018280135775011377F70FBB
:1042800041119307170022C426C21314950006C6D5
:1042900093F7E70F25809354F50185C793573400B2
:1042A000130707387604B2075207B1831395F40158
:1042B000D98FC98FB240228522449244BE854101E4
:1042C000828005EB39C42285D922A94763C6A70499
:1042D0002D47098F930755013357E4003314F40039
:1042E0009317C70013079038098FB1831377F77FAF
:1042F0005DBF01CC13573400B7070800D98FB20750
:104300007604B1831307F07F79BF1307F07F8147ED
:1043100059BF0147814741BF130755FF3317E400D9
:1043200001447DBF93D645019397C50093F6F67F70
:10433000B183138616008E071357D5011376E67FD7
:10434000FD815D8F9318350035CE138806C893071D
:10435000E00F63DD07018147139597009306F00F87
:10436000DE062581FE05558D4D8D82806355000B3F
:10437000931765000E07B337F000D98F93D8D80193
:10438000B3E7170113F777006301071013F7F7007E
:1043900091466303D7009107370700047D8F75C7E7
:1043A000130718001306F00F9376F70FE305C7FA0B
:1043B0009A07A58313959700DE062581FE05558D86
:1043C0004D8D8280B367170199EE85CF95479A0787
:1043D000A5831395970093F6F60FDE062581FE055B
:1043E000558D4D8D8280A5DBB70740001395970052
:1043F0009306F00FDE0681452581FE05558D4D8D16
:1044000082808147139597008146DE062581FE054F
:10441000558D4D8D8280A5576348F804F9473706BE
:104420008000B38707417D45598E6351F504795764
:1044300033070741130500023357E6006388A700DE
:10444000938626CAB316D600B3E8D800B337100156
:10445000D98F13F77700014815FB1397570085464E
:10446000E34807F48146A5B781468DB7938626C8F1
:104470003397D8003337E000B316D600B3D8F8002E
:10448000B367D700B3E7F800E9B7C28689B7C16759
:10449000637CF5029307F00F1307000263EBA7009C
:1044A0009717000093874766AA9788233305A7408C
:1044B000828021819717000093870765AA97882338
:1044C00061473305A7408280B7070001636DF5009F
:1044D00061819717000093872763AA978823214754
:1044E0003305A74082804181971700009387C761F9
:1044F000AA97882341473305A7408280B3C7A50008
:104500008D8B3307C50081E78D4763EDC700AA8710
:10451000637EE508942185078505A38FD7FEE3EB2D
:10452000E7FE828093763500AA8789CA94218507A1
:104530008505A38FD7FE93F63700C5BF9376C7FFD7
:10454000138606FE63F0C70683A3050083A2450019
:1045500083AF850003AFC50083AE050103AE4501FF
:1045600003A3850183A8C5019385450223A0770095
:1045700003A8C5FF23A2570023A4F70123A6E70140
:1045800023A8D70123AAC70123AC670023AE1701D4
:104590009387470223AE07FF75B7904191079105B6
:1045A00023AEC7FEE3EBD7FEE3E6E7F68280397180
:1045B0003EDA2ED232D436D63AD842DC46DE938763
:1045C000018122CC804326CA06CEAA8409C41C4C91
:1045D00099E32285FD290C4454102686228536C68F
:1045E000EF009013F2406244D244216182800111B5
:1045F00026CA4AC806CE22CC4EC652C4AA842E89E8
:1046000001C51C4D91E3F1219C4C804499E3268522
:10461000C9219717000093872761631BF402C040EC
:104620005E24A18BB1C71C48A1C7FD59294A1C446F
:1046300083450900FD17B1E91CC463DD0706228626
:10464000A94526856920FD576308F502294535A04F
:10465000971700009387475F6314F4008044C9B73D
:10466000971700009387475AE31CF4FAC0444DBFE4
:10467000A2852685192A55D97D55F2406244D24437
:104680004249B249224A056182801CC4050963D7A8
:104690000700184C63CAE700638845011C40138774
:1046A000170018C08CA361B7228626850D20E31061
:1046B00035F9D9B71C401387170018C0294798A3AC
:1046C00071B793870181AA8588436FF05FF201116A
:1046D00022CC26CA4AC806CE4EC6AA842E89328467
:1046E00001C51C4D91E3F526971700009387C7532A
:1046F0006317F406C0401C4C1CC45E24A18BC1C3CC
:104700001C48B5CF1C4808409379F90F1379F90F6D
:104710001D8D5C486346F500A2852685692C25E53C
:104720001C440505FD171CC41C401387170018C046
:10473000238037015C486388A7005E24858B81CB8A
:10474000A9476316F900A2852685B5240DEDF24030
:1047500062444A85D2444249B24905618280971732
:1047600000009387674E6314F400804469B797177D
:10477000000093876749E310F4F8C044ADBFA285F9
:104780002685212041D17D59D9B7411193870181D7
:1047900026C2844322C44AC006C62A892E8489C4FC
:1047A0009C4C99E326853526971700009387C747C9
:1047B000631BF402C0400317C40093170701C183B1
:1047C00093F68700ADEA93F6070195EEA5472320FF
:1047D000F900136707045AA47D55B240224492445D
:1047E000024941018280971700009387E7456314CF
:1047F000F4008044C9B7971700009387E740E31C93
:10480000F4FAC0444DBF918B9DC34C5889C993079E
:1048100044046384F5004A85292B232A04025E247C
:104820002322040093F7B7FD5EA41C481CC05E243D
:1048300093E787005EA41C4899EB5E2413070020D1
:1048400093F707286385E700A2854A8591295E24AE
:1048500013F717001DC35C4823240400B307F0407E
:104860001CCC1C480145B5FB8317C40013F707088F
:104870002DD793E707045EA485B7898B014791E3A1
:10488000584818C4F9BFDE25011122CC26CA06CE2D
:104890004AC84EC613F78700AA842E8479EBD84104
:1048A000634DE000B841634AE0000145F2406244D4
:1048B000D2444249B2490561828058547DD703A948
:1048C00004009396370123A0040063DB06067048BA
:1048D0005E24918B99C75C401D8E5C5899C33C4007
:1048E0001D8E5C540C50814626858297FD575A24B4
:1048F000631DF5009440F54763E8D706B7074020ED
:104900008507B3D7D700858BA5C31C482322040095
:104910001CC09317370163D80700FD576314F500D7
:104920009C4091E368C84C5823A02401BDDD930747
:1049300044046384F5002685ED2E232A0402B5B7CE
:104940000C500146854626850297FD572A86E311BD
:10495000F5F89C40B5DF75476385E70059476393D9
:10496000E70423A0240191B7136707045AA47D55D7
:1049700035BF83A90501E38A09F203A905008D8BE0
:1049800023A0350133093941014791E3D84918C4BF
:10499000E35D20F11C540C50CA864E862685829712
:1049A0006347A0005E2493E707045EA4C9B7AA99F1
:1049B0003309A940F1BF9C49A5C3011122CC06CE01
:1049C0002A8411C51C4D81E72EC62122B2459717B6
:1049D000000093876725639CF5004C408397C500D2
:1049E0009DC722856244F24005616FF0DFE99717A9
:1049F0000000938767256394F5000C44C5B79717AB
:104A0000000093876720E39BF5FC4C44C1BFF24054
:104A1000624401450561828001458280411122C4C2
:104A200006C62A844EA572A5232005002322050070
:104A3000232405002322050623280500232A050038
:104A4000232C0500214681451305C505EFB04FF520
:104A500097170000938787B25CD097170000938761
:104A6000A7B41CD497170000938787B85CD4971716
:104A700000009387E7BA00D01CD8B240224441011D
:104A8000828097050000938545F391AA411126C2C3
:104A9000130680069384F5FFB384C4024AC02E89AE
:104AA00022C406C6938544070D2E2A8401CD2320F7
:104AB000050023222501310508C41386840681459B
:104AC000EFB00FEE2285B2402244924402494101E8
:104AD00082801C4DA5E7411106C622C4970700003D
:104AE000938767FA1CD5938741819C43232405044F
:104AF00023260504232805046314F50085471CCDEF
:104B00002A84352848C022851D2808C42285052806
:104B100048C4484001469145EFF05FF0084405461F
:104B2000A545EFF0BFEF48440946C945EFF01FEF38
:104B300085471CCCB24022444101828082804111D1
:104B40009387418126C284434AC006C69C4C22C436
:104B50002A8981E72685EFF0DFF793848404804477
:104B6000DC40FD1763D607009C40B9CF8440C5BF29
:104B70000317C40039E7C1778507232204062320E1
:104B8000040023220400232404005CC4232804001E
:104B9000232A0400232C0400214681451305C40563
:104BA000EFB00FE0232A0402232C04022324040480
:104BB000232604042285B240224492440249410142
:104BC00082801304840671BF91454A85EFF01FEC83
:104BD00088C049FDB1472320F9000144E1BF797144
:104BE00022D44AD052CC56CA5AC85EC606D626D25D
:104BF0004ECE2A8AAE8A130485040149054BFD5B1B
:104C000009ECB25022544A8592540259F249624A40
:104C1000D24A424BB24B456182800444832944000E
:104C2000FD1963D409000040E1BFDE24637BFB0073
:104C30008397E40063877701A6855285829A33695A
:104C4000A90093848406E9BF1971A6DAAE8483951E
:104C5000E500A2DC86DE328463DB0500DE2423A0CF
:104C6000060093F7070885E7930700401DA030086A
:104C700036C6EF007020B246E34205FE7247BD67BC
:104C8000F98F7977BA9793B717009CC2F1BF930752
:104C900000041CC0F6506654D65401450961828058
:104CA000DE25011122CC06CE26CA4AC8898B2E8465
:104CB00089CF930774041CC01CC885475CC8F240A8
:104CC0006244D24442490561828074003000AA8463
:104CD000EFF09FF7A2452A892685012219E983175B
:104CE000C40013F7072061FFF19B93E727005EA440
:104CF000C9B797070000938707D99CD45E2408C0E2
:104D000008C893E707085EA4A2475CC8B24781CFF2
:104D10008315E4002685EF00D01811C55E24F19BB1
:104D200093E717005EA45E243369F900231624017B
:104D300079B7DDC183A7C5FF411122C406C626C2CB
:104D40001384C5FF63D307003E94AA84EF00301C90
:104D5000938701869C4381EF2322040023A0818650
:104D60002244B2402685924441016F00701A637E4E
:104D7000F40014403307D4006396E7009843DC4303
:104D8000369718C05CC0D9BFBA87D84319C3E37D32
:104D9000E4FE94433386D700631F86001040B2962A
:104DA00094C33386D700E31DC7FA10435843B29625
:104DB00094C3D8C375B76375C400B1479CC04DB7E1
:104DC0001040B306C4006316D70014435843B2968C
:104DD00014C058C0C0C369B78280011126CA938429
:104DE0003500F19806CE22CC4AC84EC6A104B14780
:104DF00063F3F404B14463E2B4042A89EF00301190
:104E00009387018698433A8439E0938741869C438F
:104E100091E781454A85252F23A2A186A6854A854B
:104E20003D27FD5963193507B1472320F9004A850D
:104E3000EF00100E29A0E3D004FCB1471CC10145CE
:104E4000F2406244D2444249B249056182801C402A
:104E5000858F63CF0702AD4663F6F6001CC03E9413
:104E600004C031A05C406313870223A0F1864A8509
:104E7000EF00100A1305B40093074400619933074B
:104E8000F5405DDF3A94898F1CC05DBF5CC3C5B738
:104E90002287404095BF130435007198E30285FCDA
:104EA000B305A4404A856525E31C35FBB5BF1C4608
:104EB000FD171CC663DA0700184E63C5E700A94753
:104EC0006394F5006FF0BF801C422E851387170096
:104ED00018C28CA38280011122CC26CA4AC84EC6B1
:104EE00052C406CE2A89AE893284B304D6007D5AD4
:104EF00063149400014509A80C204E864A85EFF002
:104F00001FFB0504E31645FFF2406244D2444249C8
:104F1000B249224A05618280357122CD26CB4AC929
:104F20004EC706CF52C556C35AC1DEDEE2DCE6DA12
:104F3000AA89AE843289368409C51C4D99E3EFF005
:104F40005FB997170000938727CE6398F40C83A46A
:104F50004900DE24A18BE5C79C48F5C393070002F6
:104F6000A304F1029307000302D22305F10222C633
:104F7000930B5002971A0000938A0ACF054C294BD5
:104F80004A841C2099C3639F770DB30C2441638E20
:104F90000C00E6864A86A6854E85EFF0DFF3FD57C6
:104FA000630FF51C9256E69636D21C206389071CC7
:104FB000FD571309140002C802CE3ECA02CCA30951
:104FC000010482D483450900154656852D27130414
:104FD0001900C24751E913F7070109C71307000277
:104FE000A309E10413F7870009C71307B002A30957
:104FF000E104834609001307A002638FE606F24727
:105000004A8481462546182093051400130707FD9E
:105010006377E60AB5CA3ECE85A897170000938746
:10502000A7C26395F40083A4890025B797170000F1
:10503000938787BDE39FF4F083A4C90019BFA685B9
:105040004E85EFF08FF419D97D55FA406A44DA4461
:105050004A49BA492A4A9A4A0A4BF65B665CD65CC8
:105060000D618280050431BF330555413315AC0015
:10507000C98F3EC82289B9B7324793064700184303
:1050800036C6634707023ACE18209307E002631D35
:10509000F70418309307A002631BF702B247090414
:1050A000138747009C433AC663C107023ECA2DA836
:1050B0003307E04093E727003ACE3EC8F1B7B38705
:1050C000670385462E84BA973DBFFD57C5B70504D3
:1050D00002CA81468147254618209305140013070C
:1050E00007FD6374E606F9F20C200D461715000063
:1050F000130505B8092511CD97170000938747B709
:105100001D8D93070004B397A700424505045D8DEC
:105110002AC80C201946171500001305A5B5130958
:1051200014002304B102C12B35C197B7FFFF938749
:1051300067ED95E74247B2471377071009CF91070C
:105140003EC69257D2973ED225BDB38767038546A8
:105150002E84BA9751B79D07E19BA107D5B7780078
:1051600097060000938666D726860C084E85970022
:105170000000E7000000FD572A8AE314F5FCDE2456
:1051800093F70704E39207EC1255C1B57800970630
:105190000000938686D426860C084E85012AE1BF3E
:1051A000797156CA9C49BA8A984522D426D24ECEE5
:1051B00052CC06D64AD05AC85EC6AA892E84B2847A
:1051C000368A63D3E700BA879CC00347340419C307
:1051D00085079CC01C4093F7070281C79C40890744
:1051E0009CC00329040013796900631A0900130B9A
:1051F0009401FD5B5C449840998F634CF9041C401A
:105200008346340493F70702B336D000A5EB1306A8
:105210003404D2854E85829AFD576303F5041C4001
:1052200011469840998B544481446397C700B384D6
:10523000E64063D3040081441C4418486354F700DB
:10524000998FBE94014969047D5B639824050145EB
:1052500009A885465A86D2854E85829A631E7501B5
:105260007D55B250225492540259F249624AD24AB0
:10527000424BB24B456182800509ADBF3307D40074
:1052800013060003A301C7040347540493871600C1
:10529000A2978906A381E7049DBF85462286D28511
:1052A0004E85829AE30E65FB050945B7797122D4D4
:1052B00026D24AD04ECE06D652CC56CA5AC8B68945
:1052C000942D930790063289AA842E841386350480
:1052D000638DF60263E2D706930780056386F618AE
:1052E00063EDD700638E062093073004638EF60AC1
:1052F000930A24042301D404C9A0930730066385CC
:10530000F60A93074006E395F6FE1C40084393F621
:10531000070893054500C5C61C410CC363D80700A8
:105320001307D002B307F040A301E404971600006E
:105330009386C694294765A8930700076382F616EB
:1053400063E5D7029307E0066389F6189307F00632
:10535000E390F6FA0C401C4313F805081385470048
:105360006307080608C39C4385A893075007E38397
:10537000F6FE930780076389F61293073007E399D7
:10538000F6F61C43D04181459386470014C383AA97
:10539000070056858D2601C53305554148C05C4040
:1053A0001CC8A301040461A81C43930A2404938627
:1053B00047009C4314C32301F4048547D5B793F6F3
:1053C00007041C410CC3B9DAC207C18781BF93F53A
:1053D000050408C3C9D99E231307F0066387E60EA8
:1053E00097160000938686892947A30104044C4040
:1053F0000CC463C5050008406D9908C099E3B28AE2
:1054000089CDB28AB3F5E702FD1AB6958C212380C7
:10541000BA00B3D5E70263F0E70CA147631EF700BB
:105420001C40858B91CB58401C4863C7E70093070D
:105430000003A38FFAFEFD1A3306564110C84E87AB
:10544000CA867000A2852685EFF09FD57D5A631D20
:10545000450B7D55B250225492540259F249624A8A
:10546000D24A424B45618280A382D5049716000040
:105470009386C6800C40084313F805081C411105AB
:10548000630D080208C313F7150001C793E5050271
:105490000CC04147B9FB0C4093F5F5FD0CC0B1B70A
:1054A0009C4193E707029CC193078007A302F40481
:1054B000970600009386C67D75BF13F8050408C3E0
:1054C000E30308FCC207C1837DBF970600009386F3
:1054D000E67A214719BFAE8735B794411C43CC49C2
:1054E00013F80608138547006306080008C39C43A9
:1054F0008CC339A008C393F606049C43F5DA8EA347
:1055000023280400B28A25BF14485686CA852685FA
:105510008299E30045F51C40898B8DE7B2474844EA
:10552000E35AF5F23E853DB785465686CA852685FF
:105530008299E30065F3050A5C443247998FE3459D
:10554000FAFEE9BF014A930A94017D5BF5B7411168
:1055500022C42A842E8523A201C806C6EFC0FFC339
:10556000FD576317F500938741C89C4391C31CC046
:10557000B240224441018280411122C42E8483958D
:10558000E50006C67922634905007C48AA977CC8D5
:10559000B2402244410182805E247D777D17F98FDD
:1055A0005EA4FDB7DE25011122CC26CA4AC84EC62C
:1055B00006CE93F70710AA842E843289B68991C744
:1055C0008395E5008946014609225E247D777D1793
:1055D000F98F5EA48315E4006244F240CE864A86C9
:1055E000B24942492685D244056125A8411122C409
:1055F0002E848395E50006C6C928FD575A24631AF0
:10560000F500FD77FD17F98F5EA4B24022444101F9
:1056100082808567D98F5EA468C8C5BF8395E50081
:1056200005A8411122C42A842E85B285368623A27C
:1056300001C806C6EFC09FB2FD576317F5009387F8
:1056400041C89C4391C31CC0B240224441018280A6
:10565000411122C42A842E8523A201C806C6C52072
:10566000FD576317F500938741C89C4391C31CC045
:10567000B240224441018280411122C42A842E85F5
:10568000B28523A201C806C6C920FD576317F500DD
:10569000938741C89C4391C31CC0B240224441013E
:1056A0008280411122C42A842E8523A201C806C605
:1056B0005D20FD576317F500938741C89C4391C354
:1056C0001CC0B240224441018280411122C42A847C
:1056D0002E85B285368623A201C806C65920FD57FD
:1056E0006317F500938741C89C4391C31CC0B24027
:1056F00022444101828093F5F50F2A966314C50078
:10570000014582801C21E38EB7FE0505C5BF82805E
:105710008280411122C42A842E85B285368623A236
:1057200001C806C6A920FD576317F500938741C835
:105730009C4391C31CC0B240224441018280930724
:10574000800523A2F1C87D5582809307800523A29E
:10575000F1C87D5582809307800523A2F1C80145D9
:1057600082809307800523A2F1C87D55828093072C
:10577000800523A2F1C87D5582800000537973749F
:10578000656D436C6B3A25640D0A000043686970CF
:1057900049443A253038780D0A00000043616C69AD
:1057A0006272617474696F6E5F56616C203A202575
:1057B000640A0000CDCC4C3D6666663F0000F043B5
:1057C0009A9999999999A93FCDCCCCCCCCCCEC3F66
:1057D000696E2074696D31206972712000000000CB
:1057E0000000804000000000000000000000E03FDA
:1057F0000000000000003440000030411D130F1372
:105800000213F412E612D712C812B912AA129A128F
:105810008A127A126A12591248123712251213127A
:105820000112EE11DB11C811B511A1118D11791101
:1058300064114F113A1125110F11F910E310CC101A
:10584000B5109E1087106F1057103F1026100D10C6
:10585000F40FDB0FC20FA80F8E0F740F590F3F0FFD
:10586000240F090FED0ED20EB60E9A0E7E0E620EAA
:10587000460E290E0C0EF00DD30DB60D980D7B0DB6
:105880005E0D400D220D050DE70CC90CAB0C8D0C07
:105890006F0C510C330C150CF70BD90BBB0B9C0B7D
:1058A0007E0B600B420B240B060BE80ACA0AAD0AFA
:1058B0008F0A710A540A360A190AFC09DF09C2095B
:1058C000A50988096C094F0933091709FB08DF0886
:1058D000C308A8088D08720857083C082108070863
:1058E000ED07D307B907A00786076D0754073C07E4
:1058F00023070B07F306DB06C406AD0696067F06F4
:10590000680652063C0626061006FB05E605D1058C
:10591000BC05A70593057F056B05580545053205B0
:105920001F050C05FA04E804D604C404B304A1045A
:1059300090047F046F045F044E043E042F041F0490
:1059400010040104F203E303D503C703B903AB0357
:105950009D0390038203750368035C034F034303B5
:1059600036032A031F0313030703FC02F102E602B6
:10597000DB02D102C602BC02B202A7029E0294025E
:105980008A02810277026E0265025C0254024B02B7
:1059900042023A0232022A0222021A0212020B02C6
:1059A0000302FC01F401ED01E601DF01D801D2019F
:1059B000CB01C401BE01B801B101AB01A5019F013A
:1059C000990194018E01880183017D0178017301A1
:1059D0006E01690163015E015A0155015001000029
:1059E00000007A440AD7A33B25640A0025640D0A07
:1059F000000000000000803F0000C842000070412D
:105A0000CDCC4C3FB6D2FFFFA8D1FFFFA8D1FFFFFE
:105A1000A6D1FFFFAED1FFFFAED1FFFF74D1FFFFD4
:105A2000A6D1FFFFAED1FFFF74D1FFFFAED1FFFFC4
:105A3000A6D1FFFFA2D2FFFFA2D2FFFFA2D2FFFF9B
:105A400074D1FFFF88DEFFFFAEDDFFFF82DEFFFFC8
:105A5000B6DDFFFF82DEFFFF7CDDFFFF82DEFFFFA2
:105A6000B6DDFFFFAEDDFFFFAEDDFFFF7CDDFFFF3C
:105A7000B6DDFFFFBCDDFFFFBCDDFFFFBCDDFFFFD0
:105A80007CDDFFFF6EDDFFFF6EDDFFFF42DEFFFF0F
:105A90001EDFFFFF42DEFFFF3CDDFFFF42DEFFFFB8
:105AA0001EDFFFFF6EDDFFFF6EDDFFFF3CDDFFFF52
:105AB0001EDFFFFF7CDDFFFF7CDDFFFF7CDDFFFFE6
:105AC0003CDDFFFF96E1FFFFE4E0FFFFE4E0FFFFC6
:105AD000E2E0FFFFE8E0FFFFE8E0FFFFB8E0FFFFE4
:105AE000E2E0FFFFE8E0FFFFB8E0FFFFE8E0FFFFD4
:105AF000E2E0FFFF84E1FFFF84E1FFFF84E1FFFFBD
:105B0000B8E0FFFF000102020303030304040404DE
:105B10000404040405050505050505050505050539
:105B20000505050506060606060606060606060619
:105B30000606060606060606060606060606060605
:105B400006060606070707070707070707070707E9
:105B500007070707070707070707070707070707D5
:105B600007070707070707070707070707070707C5
:105B700007070707070707070707070707070707B5
:105B80000707070708080808080808080808080899
:105B90000808080808080808080808080808080885
:105BA0000808080808080808080808080808080875
:105BB0000808080808080808080808080808080865
:105BC0000808080808080808080808080808080855
:105BD0000808080808080808080808080808080845
:105BE0000808080808080808080808080808080835
:105BF0000808080808080808080808080808080825
:105C00000808080800000000000000000000000074
:105C10000000000000000000000000000000000084
:105C20000000000000000000000000000000000074
:105C30000000000000000000000000000000000064
:105C40000000000000000000000000000000000054
:105C50000000000000000000000000000000000044
:105C600000000000232D302B20000000686C4C0049
:105C70006566674546470000303132333435363784
:105C80003839414243444546000000003031323348
:105C90003435363738396162636465660000000068
:105CA00000000000000000000102030406070809CC
:105CB00000000000010203040102030406070809B2
:105CC00000000000000000000000000000E8038C5D
:105CD000051400A406DC05A00564008C050A00017B
:105CE00000140014004600320028000A003C001096
:105CF0000E000000534C111111111111110100017E
:105D000000160000000000000300000080250000D5
:105D10000000000000000000000000000000000083
:105D200000000000040000008025000000000000CA
:105D30000000000000000000000000000000000063
:105D4000245C0000445C0000045C000000000000D3
:105D50000000000000000000000000000000000043
:105D60000000000000000000000000000000000033
:105D70000000000000000000000000000000000023
:105D80000000000000000000000000000000000013
:105D90000000000000000000000000000000000003
:105DA000006CDC0202040608880500200000403F69
:085DB0009C0000209C00002073
:00000001FF
